:020000000150AD
:02000B00019D55
:02001B0021D6EC
:02002300217F3B
:1000500075900075B00175816F75200175892175E6
:100060008DF3D28E7598C0438780C299C298D2AB67
:10007000D2ACD29CD28CD28CD2A9D2AFD2B97530AC
:100080000175310175213F752800752964752212AB
:10009000752334752456315A7528000196C0E0C086
:1000A000D0C000D5300B753064D53105753103B241
:1000B00030758CFAD520037520060090015CE52090
:1000C00014C31392D52422F8E630D504540F8003CC
:1000D00054F0C493A820759000B80110D2B4C2B2F5
:1000E000A20D92E03030643045618066B80210D2D3
:1000F000B2C2B3A20C92E030305130444E8053B8BB
:100100000310D2B3C2B1A20B92E030303E30433B79
:100110008040B80410D2B1C2B7A20A92E030302BAE
:10012000304228802DB80510D2B7C2B5A20992E09E
:10013000303018304115801AB80610D2B5C2B4A2BA
:100140000892E03030053040028007F59085293272
:10015000C23100D000D0D0D0E0320022FC60DAF210
:1001600066B6BEE0FEF6EE3E9C7A9E00FD61DBF3D5
:1001700067B7BFE1FFF7EF3F9D7B9F8F0002C6C0CF
:10018000E0C299C298209A427404B52706E599F511
:1001900022803E7405B52706E599F5238033740661
:1001A000B52706E599F52480287407B52706E59953
:1001B000F529801D7408B52706E599F5218012748C
:1001C00009B52704E599F5288007E599F527D0E0DA
:1001D000320527D0E03230310132D53205D23175C7
:0301E0009000325A
